:020000040000FA
:2B000000FFFF62FF2500FFFFFFFFFFFFFFFFFFFFFFFFFFFFFFFFFFFFFFFFFFFFFFFFFFFFFFFFFFFFFFFFFFFFFFFFFF76
:2B002B00C01D96611986C11D96C17507777007D71DBC010000000070DDC11D8661195C7758866119DC6118DC6100F30C
:2B005600A0100EE11004A1100EA12884422884A2100A0100000000280AA11004E1108A423804E1100A41100A4100831B
:2B008100000000000000000000000000000000000000000000000000000000000000000000000000000000000080E7ED
:2B00AC00000000000000000000000000000000000000000000000000000000000000000000000000000000000080E7C2
:2B00D700000008808000000008000000000000000000000000000000000000008000000020008001000000000000D5F8
:2B010200000020200000000004000000000000000000000000000000000000002400000018002000000000000000F83A
:2B012D00000000000000000000000000000000000000000000000000000000000000000000000000000000000080E740
:2B015800060000000000000000000000000000000000000000000000000000000000000000000000000000000080E115
:2B018300000000000000000000000000000000000000000000000000000000000000000000000000000000000080E7EA
:2B01AE00180000000000000000000000000000000000000000000000000000000000000000000000000000000080FF8F
:2B01D900000000000000000000000000000000000000000000000000000000000000000000000000000000000080E794
:2B020400000000000000000000000000000000000000000000000000000000000000000000000000000000000080E768
:2B022F00000000000000000000800000000000000000000000000000000000000000000000000000000000000000EF35
:2B025A00000000000000000000000000000000000000000000000000000000000000000000000000000000000080E712
:2B028500000000000000000000000000000000000000000000000000000000000000000000000000000000000080E7E7
:2B02B000060000000000000000000000000000000000000000000000000000000000000000000000000000000080E1BC
:2B02DB00000000000000000000000000000000000000000000000000000000000000000000000000000000000008EF01
:2B030600000000000000000000000000000000000000000000000000000000000000000000000000000000000080E765
:2B033100000000000040000000000200000000000000000000000000000000000000000000000000000000000080815E
:2B035C00000000000010000000000300000000000000000000000000000000000000000000000000000000000080C51E
:2B0387000000000000020800000000A0000000000000000000000000000000000000000000000000000000000000EDB4
:2B03B200020000000000000000000008000000000000000000000000000000000000000000000000000000000088E5A9
:2B03DD00020000000000000000000000000000000000000000000000000000000000000000000000000000000080E58E
:2B040800040000000000000000000000000000000000000000000000000000000000000000000000000000000080E362
:2B0433000200000000020800000000B8020000000000000000000000000000000000000000000000000000000080F464
:2B045E00020000000000000000000000000000000000000000000000000000000000000000000000000000000080E50C
:2B048900020000000000000000000000000000000000000000000000000000000000000000000000000000000008ED51
:2B04B400800008800008800008800008800008800008000000000020000220000220000220000220000220000280E7BA
:2B04DF00800008800008800008800008800008800008000000000020000220000220000220000220000220000280E78F
:2B050A00000000000000100000000100000000000000000000000000000000000000000000000000000000000080E64F
:2B053500020000000026000000E02000000000000000000000000000000000000000000000000000000000000000CDA6
:2B056000020000000018000000800000000000000000000000000000000000000000000000000000000000000008FCD2
:2B058B0004000000001C040000400B00000000000000000000000000000000000000000000000000000000000008C509
:2B05B600020000000018000000800000000000000000000000000000000000000000000000000000000000000008FC7C
:2B05E100020000000018000000001100000000000000000000000000000000000000000000000000000000000088E458
:2B060C00020000000000000000000100000000000000000000000000000000000000000000000000000000000080F44C
:2B063700000000000000000000801200000000000000000000000000000000000000000000000000000000000000CC3A
:2B066200000000000000000000000000000000000000000000000000000000000000000000000000000000000080E706
:2B068D0000000000000000000060210000000000000000000000000000000000000000000000000000000000008094AD
:2B06B800020000000000000000000100000000000000000000000000000000000000000000000000000000000008FC10
:2B06E300020000000000000000C00500000000000000000000000000000000000000000000000000000000000000F82D
:2B070E00040000000000000000000000000000000000000000000000000000000000000000000000000000000080E359
:2B073900020000000000000000808200000000000000000000000000000000000000000000000000000000000000C7CA
:2B076400020000000000000000800000000000000000000000000000000000000000000000000000000000000000EDFB
:2B078F00020000000000000000802300000000000000000000000000000000000000000000000000000000000088D43E
:2B07BA00000000000000000000000100000000000000000000000000000000000000000000000000000000000080F69D
:2B07E500000000000036020000E02000000000000000000000000000000000000000000000000000000000000000DCD5
:2B081000000000000010000000800000000000000000000000000000000000000000000000000000000000000000FE2F
:2B083B0002000000005C000000400500000000000000000000000000000000000000000000000000000000000000ED02
:2B086600020000000000000000800000000000000000000000000000000000000000000000000000000000000088E578
:2B089100040000000008020000008300000000000000000000000000000000000000000000000000000000000088DA49
:2B08BC00020000000008080000000100000000000000000000000000000000000000000000000000000000000088FC7A
:2B08E700020000000038000000802200000000000000000000000000000000000000000000000000000000000008FE04
:2B091200020000000010000000000100000000000000000000000000000000000000000000000000000000000080E542
:2B093D0000000000002E020000E02000000000000000000000000000000000000000000000000000000000000080C51A
:2B096800000000000088000000800400000000000000000000000000000000000000000000000000000000000000A3B5
:2B099300000000000014000000400300000000000000000000000000000000000000000000000000000000000080C59D
:2B09BE00000000000008000000800001000000000000000000000000000000000000000000000000000000000080F70E
:2B09E900020000000030010000000300000000000000000000000000000000000000000000000000000000000008ECB9
:2B0A1400020000000010000000000300000000000000000000000000000000000000000000000000000000000008CFCB
:2B0A3F00020000000028100000800200000000000000000000000000000000000000000000000000000000000008FDCB
:2B0A6A00020000000010000000000000000000000000000000000000000000000000000000000000000000000008FC4B
:2B0A950000000000002E020000602100000000000000000000000000000000000000000000000000000000000000DCA9
:2B0AC000000000000048000000000100000000000000000000000000000000000000000000000000000000000000BA08
:2B0AEB00000000000034000000C00B00000000000000000000000000000000000000000000000000000000000080EF72
:2B0B1600000000000008000000000000000000000000000000000000000000000000000000000000000000000000EFBD
:2B0B4100000000000010100000801000000000000000000000000000000000000000000000000000000000000000EFEA
:2B0B6C00020000000010010000800000000000000000000000000000000000000000000000000000000000000088F54E
:2B0B9700020000000008000000801300000000000000000000000000000000000000000000000000000000000008DFAF
:2B0BC200020000000000000000000000000000000000000000000000000000000000000000000000000000000008ED11
:2B0BED00020000000026020000602100000000000000000000000000000000000000000000000000000000000008DE4C
:2B0C1800000000000000100000000500000000000000000000000000000000000000000000000000000000000080A27A
:2B0C430000000000003C000000C00300000000000000000000000000000000000000000000000000000000000080E720
:2B0C6E00000000000018000000000001000000000000000000000000000000000000000000000000000000000000EE54
:2B0C9900000000000000040000800200000000000000000000000000000000000000000000000000000000000000C9E1
:2B0CC400000000000018000000800200000000000000000000000000000000000000000000000000000000000080D417
:2B0CEF00020000000018000000800300000000000000000000000000000000000000000000000000000000000008CF66
:2B0D1A00020000000000000000000000000000000000000000000000000000000000000000000000000000000008EDB7
:2B0D4500020000000036020000602100000000000000000000000000000000000000000000000000000000000008CFF1
:2B0D7000020000000090000000001100000000000000000000000000000000000000000000000000000000000088EC41
:2B0D9B0000000000001C000000C00300000000000000000000000000000000000000000000000000000000000080C509
:2B0DC600000000000000000000000000000000000000000000000000000000000000000000000000000000000080E79B
:2B0DF100000000000028010000800001000000000000000000000000000000000000000000000000000000000080D4D9
:2B0E1C00000000000008000000801000000000000000000000000000000000000000000000000000000000000080E6AD
:2B0E4700020000000038100000800100000000000000000000000000000000000000000000000000000000000080D75E
:2B0E7200020000000010000000000100000000000000000000000000000000000000000000000000000000000008ED4D
:2B0E9D0004000000002E020000E02000000000000000000000000000000000000000000000000000000000000008C925
:2B0EC800020000000008000000800400000000000000000000000000000000000000000000000000000000000008A9C0
:2B0EF300020000000054000000400100000000000000000000000000000000000000000000000000000000000008A98C
:2B0F1E00020000000008000000802000000000000000000000000000000000000000000000000000000000000080E797
:2B0F4900000000000010020000000100000000000000000000000000000000000000000000000000000000000080E505
:2B0F7400000000000010080000000300000000000000000000000000000000000000000000000000000000000080CDEA
:2B0F9F000000000000280000008000000000000000000000000000000000000000000000000000000000000000A0E7F8
:2B0FCA001C000000000000000000000000000000000000000000000000000000000000000000000000000000007884E4
:2B0FF500000000000000000000000000000000000000000000000000000000000000000000000000000000000080E76A
:2B102000800008800008800008800008800008800008000000000020000220000220000220000220000220000280E742
:2B104B00800008800008800008800008800008800008000000000020000220000220000220000220000220000280E717
:2B107600000000004022000000000000000000000000000000000000000000000000000000000000000000000080E18C
:2B10A100000000004000000000000000000000000000000000000000000000000000000000000000000000000080E381
:2B10CC000000000000000000000040002000040000000000000000000000000000000000000000000000000000808392
:2B10F700000000000000000000800000000000000080000000000000000000000000000000000000000000000080EF5F
:2B112200000000004022000000000000200004000080000000000000000000000000000000000000000000000000811B
:2B114D00000000000020100000400401000000000000000000000000000000000000000000000000000000000080C1C1
:2B117800000000000000000000000000000000000000000000000000000000000000000000000000000000000080E7E5
:2B11A300000000000008080000004000000000000000000000000000000000000000000000000000000000000000E3EE
:2B11CE00000000000000040000408000000000000000000000000000000000000000000000000000000000000080AB07
:2B11F900000000000000010000000000000000000000000000000000000000000000000000000000000000000080E664
:2B122400000000000000000000000000000000000000000000000000000000000000000000000000000000000080E738
:2B124F00000000000000000000000000000000000000000000000000000000000000000000000000000000000080E70D
:2B127A00000000000000000000000000000000000000000000000000000000000000000000000000000000000080E7E2
:2B12A500020000000000000000000100000000000000000000000000000000000000000000000000000000000080F4A7
:2B12D000000000000000000000000000000000000000000000000000000000000000000000000000000000000080E78C
:2B12FB00000000000000000000000000000000000000000000000000000000000000000000000000000000000080E761
:2B132600000000000000080000800000000000000000000000000000000000000000000000000000000000000000E72D
:2B135100000000000000000000000000000000000000000000000000000000000000000000000000000000000080E70A
:2B137C00000000000000000000000000000000000000000000000000000000000000000000000000000000000080E7DF
:2B13A700020004000000000000000000000000000000000000000000000000000000000000000000000000000080A5F0
:2B13D200000000000000000000000000000000000000000000000000000000000000000000000000000000000080E789
:2B13FD00000000000000000000000000000000000000000000000000000000000000000000000000000000000080E75E
:2B142800000000000000000400000000000000000000000000000000000000000000000000000000000000000080A372
:2B145300000000020000000000000000000000000000000000000000000000000000000000000000000000000080E507
:2B147E00000000000000000000000000000000000000000000000000000000000000000000000000000000000080E7DC
:2B14A900000000000000000000000000000000000000000000000000000000000000000080000000000000000088EF21
:2B14D400040000000000000000000000000000000000000000000000000000000000000000000000000000000090F267
:2B14FF00000000000000000001000000000000000000000000000000000000000400000000000000000000000080B38A
:2B152A00040014000000000001000000000000000000000000000000000000001040000020000000000000000090D4A9
:2B1555000000000000000001000000000000000000000000000000000000000000000000400000000000000000A090FA
:2B158000000000000000000000000000000000000000000000000000000000000000000000000000000000000080E7D9
:2B15AB000000200000000002000000000000000000000000000000000000000000C0000000010000000000000000A290
:2B15D600000000000000000200000000000000000000000000000000000000000000000000000000000000000080C5A3
:2B160100200002000000200200400000000880400020000000000008022000000088040000008000020000020000CB4D
:2B162C00220000000000200008400000000000400020000000000008000000000000000000000000000000000080C75A
:2B165700000010000000000000000000000000000000000000000000000000000000000000000400000000000008BA92
:2B168200000000000000000000000000000880000000000000000000022000000000040000000000020000020008EB98
:2B16AD00000002000000000208000000000000000000000000000000000000000088000000008400000000000088A1D1
:2B16D800000000000000000000000000000000000000000000000000000000000000000000000000000000000008EFF0
:2B170300020000000000000000000000000000000000000000000000000000000000000000000000000000000080E554
:2B172E00800008800008800008800008800008800008000000000020000220000220000220000220000220000280E72D
:2B175900800008800008800008800008800008800008000000000020000220000220000220000220000220000280E702
:2B178400000000000000000100000000000000000000000000000000000000000000000000000000000000000080F6C3
:2B17AF00000016020000E02000000000000000000000000000000000000000000058080000000000000000000080AB6C
:2B17DA00020010000000800000000000000000000000000000000000000000000040000000000000000000000088B0DA
:2B1805000200BC000000400B000000000000000000000000000000000000000000F00200000000000000000000089025
:2B183000020000080000800001000000000000000000000000000000000000000000080000000000000000000088F57D
:2B185B00020008000000000100000000000000000000000000000000000000000020000000000000000000000088D6D9
:2B188600000028000000008100000000000000000000000000000000000000000020000000000000000000000000F678
:2B18B100000018000000800200000000000000000000000000000000000000000060040000000000000000000080B6D8
:2B18DC00000000000000000000000000000000000000000000000000000000000000000000000000000000000080E77A
:2B1907000000160200006021000000000000000000000000000000000000000000580800D8080000000000000000E7F5
:2B193200020050000000000100000000000000000000000000000000000000000040010040010000000000000008A904
:2B195D0002003C000000C009000000000000000000000000000000000000000000F0000070000000000000000008CF21
:2B198800040000000000000200000000000000000000000000000000000000000000040080000000000000000010D4C6
:2B19B3000200080100008000000000000000000000000000000000000000000000200000A0000000000000000088EC4A
:2B19DE00020028000000800000000000000000000000000000000000000000000020000020000000000000000008CF1D
:2B1A0900020038000000800101000000000000000000000000000000000000000060200060400000000000000008BF0F
:2B1A3400000010000000000100000000000000000000000000000000000000000040000040000000000000000080E78F
:2B1A5F0000000E020000E020000000000000000000000000000000000000000000380800B8080000000000000000E765
:2B1A8A00000088000000800000000000000000000000000000000000000000000020000020010000000000000000E602
:2B1AB5000200340000004003010000000000000000000000000000000000000000D0020050000000000000000088FFE3
:2B1AE0000200080800008000000000000000000000000000000000000000000000200800A0000000000000000088ED0C
:2B1B0B000400300000000011000000000000000000000000000000000000000000400000C0000000000000000010D189
:2B1B3600020010010000000101000000000000000000000000000000000000000040000040000000000000000008FCEB
:2B1B61000200080000008002000000000000000000000000000000000000000000200400204000000000000000088BB6
:2B1B8C00020010000000000000000000000000000000000000000000000000000040000040000000000000000008FC98
:2B1BB70000000E0200006021000000000000000000000000000000000000000000380800B8080000000000000080FEF4
:2B1BE200000048000000000100000000000000000000000000000000000000000020020020000000000000000000B895
:2B1C0D00000034000000C005000000000000000000000000000000000000000000D00000D00200000000000000008B86
:2B1C3800020008000000002000000000000000000000000000000000000000000020200020000000000000000088C7A8
:2B1C63000200100100008002000000000000000000000000000000000000000000C00000C0040000000000000088D3E2
:2B1C8E000400300000008000000000000000000000000000000000000000000000C0000040040000000000000090CD16
:2B1CB9000200280000008013000000000000000000000000000000000000000000200000A0000000000000000088FDFE
:2B1CE400020010000000000100000000000000000000000000000000000000000040000000000000000000000008A9D1
:2B1D0F0002000E020000E020000000000000000000000000000000000000000000380800D80800000000000000888B64
:2B1D3A000000081000008000000000000000000000000000000000000000000000200100400000000000000000809075
:2B1D65000000140000004005000000000000000000000000000000000000000000D00000700100000000000000008039
:2B1D9000000008000000802000000000000000000000000000000000000000000020040080000000000000000000C319
:2B1DBB00000010080000000300000000000000000000000000000000000000000040000020000000000000000008A3D7
:2B1DE600020010000000000100000000000000000000000000000000000000000040000020000000000000000080835C
:2B1E1100020028080000801200000000000000000000000000000000000000000020200060080000000000000080803A
:2B1E3C00020010000000000000000000000000000000000000000000000000000040000000000000000000000080B0F9
:2B1E670002000E0200006021000000000000000000000000000000000000000000380800D80800000000000000809A83
:2B1E92000000080000000041000000000000000000000000000000000000000000200000400000000000000000889460
:2B1EBD000000B4000000C003000000000000000000000000000000000000000000504000F0400000000000000000CDF6
:2B1EE8000000080800000020000000000000000000000000000000000000000000A0000000000000000000000080C7B8
:2B1F13000000100000008000000000000000000000000000000000000000000000C00000200400000000000000809C13
:2B1F3E00000030000000800000000000000000000000000000000000000000000040200020400000000000000000DA2E
:2B1F69000200080000008041000000000000000000000000000000000000000000200000E0000000000000000088BC3E
:2B1F9400020000000000000000000000000000000000000000000000000000000000000000000000000000000008ED2B
:2B1FBF000200160200006021000000000000000000000000000000000000000000580800D8080000000000000088EDA7
:2B1FEA00020010100000000100000000000000000000000000000000000000000040000040000000000000000008FD24
:2B20150000001C000000C00B000000000000000000000000000000000000000000704000F00200000000000000808710
:2B204000000000000000000001000000000000000000000000000000000000000080000000000000000000000000F7FD
:2B206B000000080800008000000000000000000000000000000000000000000000A00000A0040000000000000080EB0B
:2B209600000008000000808000000000000000000000000000000000000000000020200020040000000000000080CB68
:2B20C1000200380800008003000000000000000000000000000000000000000000600000E0000000000000000088E582
:2B20EC00020000000000000100000000000000000000000000000000000000000800020040000000000000000088BA3A
:2B211700040016020000E02000000000000000000000000000000000000000800FD80000B8080000000000000010FA50
:2B214200020090000000800000000000000000000000000000000000000000008660000020000000000000000008DE74
:2B216D0002003C000000400900000000000000000000000000000000000000000950080050010000000000000088DFA7
:2B2198000200000800008002000000000000000000000000000000000000000006402000A0000000000000000008EF93
:2B21C3000000280000000001000000000000000000000000000000000000000040E0000040000000000000000080FAEE
:2B21EE000000080100000001000000000000000000000000000000000000000000C0000040000000000000000080FF3D
:2B2219000800180000008000010000000000000000000000000000000000000006000000200800000000000000C0E625
:2B2244000C0000000000000000000000000000000000000000000000000000000000000000000000000000000090FAD9
:2B226F00000000000000000000000000000000000000000000000000000000000000000000000000000000000080E7DD
:2B229A00800008800008800008800008800008800008000000000020000220000220000220000220000220000280E7B6
:2B22C500800008800008800008800008800008800008000000000020000220000220000220000220000220000280E78B
:2B22F000000000080000200208000000000000000000000000000000000000000008200088000000000000000080C59C
:2B231B00000000000000000000000000000000000000000000000000000000000000000000000000000000000080E730
:2B234600200000200000400002000000000000000400000000000000000000000000000000000108800000000080D20B
:2B237100000000000000000008008000000000000000000000000000000000024000084000020000002000000000ED20
:2B239C002000082A0000600202008000000000000400000000000000000000024208204088020108802000000080DAA3
:2B23C700000010000000801000000000000000000000000000000000000000000000000000000000000000000000FF4C
:2B23F200000000000000008000000000000000000000000000000000000000000180000000200000000000000000DEC1
:2B241D00000000000000408000000000000000000000000000000000000000000000000020600000000000000080EDE7
:2B244800000000020000000000000000000000000000000000000000000000000000000000000000000000000080E502
:2B247300000000040000000000000000000000000000000000000000000000000000400010000000000000000048FEA4
:2B249E00020000100000004000000000000000000000000000000000000000000010180000000000000000000080F821
:2B24C9000000000000000000000000000000000000000000000000000000000000000000000000000000000000C0A385
:2B24F400000000040000000000000000000000000000000000000000000000000000000000000000000000000080E356
:2B251F00000000000000000000000000000000000000000000000000000000000000000000000000000000000080E72A
:2B254A00000000000000000000000000000000000000000000000000000000000000000010000000000000000008FE50
:2B257500000000000000000000000000000000000000000000000000000000000010000000000000000000000080F6B5
:2B25A000100000000000000800000000000000000000000000000000000000000000000000000000000000000000F701
:2B25CB00000000000000000000000000000000000000000000000000000000000000080000000000000000000080EF6E
:2B25F600000000000000000000000000000000000000000000000000000000000000000000000000000000000080E753
:2B262100000000000000000000000000000000000000000000000000000000000000000000000004000000000080A763
:2B264C00100000000000000000000000000000000000000000000000000000000000000000000000000000000080F7DC
:2B267700000000000000000000000000000000000000000000000000000000000000000000001000000000000080E6C2
:2B26A200020000000000000000000000000000000000000000000000000000000000000000000000000000000080E5A6
:2B26CD00000000000000000000000000000000000000000000000000000000000000000000000000000000000080E77B
:2B26F800000000000000000000000000000000000000000000000000000000000000000000000000000000000080E750
:2B272300000000000000000000000000000000000000000000000000000000000000000000000000000000000080E724
:2B274E000000000000000000000000000000000000000000000000000000000000000000000000000000000000C0A3FD
:2B277900000000000000000010000000000000000000000000000000000000000000000000000000000000000080F6AF
:2B27A4001000000000000000000000000000000000000000000000000000000000000000000000000000000000C0B387
:2B27CF00000000000000000000000000000000000000000000000000000000000000000000000000000000000080E778
:2B27FA00000000000000000000000000000000000000000000000000000000000000000000000000000000000080E74D
:2B2825000000000000000000A0000000000000000000000000000000000000000000000000000800000000000080C59B
:2B285000000000000000000000000000000000000000000000000000000000000000000000000000000000000080E7F6
:2B287B00000000000000000002090880000000000000000000000000000000000000800020000002000000000000C439
:2B28A600020000000000000000000000000000000000000000000000000000000000800000000000000000000088E518
:2B28D100020000000000000000000000000000000000000000000000000000000000000000000000000000000008EDE5
:2B28FC00040000000000000000000880000000000000000000000000000000000000000000000000000000000090F2A3
:2B292700020000000000000002090000000000000000000000000000000000000000000020000002000000000008C688
:2B295200020000000000000000000000000000000000000000000000000000000000000000000000000000000008ED63
:2B297D00020000000000000000000000000000000000000000000000000000000000000000000000000000000008ED38
:2B29A800800008800008800008800008800008800008000000000020000220000220000220000220000220000280E7A1
:2B29D300800008800008800008800008800008800008000000000020000220000220000220000220000220000280E776
:2B29FE00000000000000000010000000000000000000000000000000000000000000000000000400000000000080B268
:2B2A290000000000000000000E020000000000000000000000000000000000000000000000808300000000000080BE31
:2B2A5400020000000000000088000000000000000000000000000000000000000000000000000200000000000008C7FC
:2B2A7F00020000000000000014000000000000000000000000000000000000000000000000000504000000000008A95C
:2B2AAA0002000000000000000810000000000000000000000000000000000000000000000000020400000000008897C2
:2B2AD500020000000000000030000000000000000000000000000000000000000000000000000C000000000000889A76
:2B2B0000000000000000000010080000000000000000000000000000000000000000000000000400000000000080BA54
:2B2B2B00000000000000000008000000000000000000000000000000000000000000000000008A00000000000080C5A8
:2B2B5600000000000000000000000000000000000000000000000000000000000000000000000000000000000080E7ED
:2B2B8100000000000000000016020000000000000000000000000000000000000000000000808500000000000000C14B
:2B2BAC00000000000000000090000000000000000000000000000000000000000000000000002400000000000000B09A
:2B2BD70002000000000000001C000000000000000000000000000000000000000000000000000700000000000088C363
:2B2C0200020000000000000000100000000000000000000000000000000000000000000000000000000000000008FD90
:2B2C2D00020000000000000028000000000000000000000000000000000000000000000000000A01000000000008F54A
:2B2C58000200000000000000080800000000000000000000000000000000000000000000000002040000000000888F22
:2B2C83000000000000000000180000000000000000000000000000000000000000000000000006000000000000009870
:2B2CAE00000000000000000000000000000000000000000000000000000000000000000000000000000000000080E794
:2B2CD900000000000000000016020000000000000000000000000000000000000000000000808500000000000000C1F2
:2B2D0400000000000000000010000000000000000000000000000000000000000000000000001400000000000080B34D
:2B2D2F0002000000000000005C000000000000000000000000000000000000000000000000000F000000000000808FFD
:2B2D5A00020000000000000020000000000000000000000000000000000000000000000000000800000000000088CFCD
:2B2D8500040000000000000008000000000000000000000000000000000000000000000000000200000000000088C1CC
:2B2DB000020000000000000008000000000000000000000000000000000000000000000000000201000000000088D78C
:2B2DDB00020000000000000018010000000000000000000000000000000000000000000000000E000000000000089309
:2B2E0600020000000000000010000000000000000000000000000000000000000000000000000400000000000080B05B
:2B2E310000000000000000000E020000000000000000000000000000000000000000000000808300000000000080BE25
:2B2E5C00000000000000000008000000000000000000000000000000000000000000000000001200000000000000CC65
:2B2E8700000000000000000054000000000000000000000000000000000000000000000000000D00000000000000A718
:2B2EB200020000000000000028000000000000000000000000000000000000000000000000000A00000000000008E5D4
:2B2EDD00020000000000000010000000000000000000000000000000000000000000000000000400000000000008B8F4
:2B2F0800040000000000000010000000000000000000000000000000000000000000000000000401000000000090B73E
:2B2F3300020000000000000008010000000000000000000000000000000000000000000000000A00000000000008C690
:2B2F5E00020000000000000010000000000000000000000000000000000000000000000000000400000000000008B872
:2B2F890002000000000000000E020000000000000000000000000000000000000000000000808300000000000008B44C
:2B2FB400000000000000000008000000000000000000000000000000000000000000000000002200000000000000CFF9
:2B2FDF00000000000000000034100000000000000000000000000000000000000000000000000500000000000080D12D
:2B300A00000000000000000008000000000000000000000000000000000000000000000000000200000000000000CDC4
:2B303500000000000000000010100000000000000000000000000000000000000000000000000C01000000000088BA01
:2B306000020000000000000010000000000000000000000000000000000000000000000000000404000000000008F82B
:2B308B00020000000000000028020000000000000000000000000000000000000000000000000200000000000010FEDE
:2B30B600020000000000000000000000000000000000000000000000000000000000000000000400000000000008A938
:2B30E100020000000000000016020000000000000000000000000000000000000000000000808300000000000088AD72
:2B310C00000000000000000010000000000000000000000000000000000000000000000000000200000000000008DCA2
:2B31370000000000000000007C000000000000000000000000000000000000000000000000002D000000000000808FB5
:2B316200000000000000000000000000000000000000000000000000000000000000000000004200000000000080C1BF
:2B318D000000000000000000280400000000000000000000000000000000000000000000000004000000000000008D5A
:2B31B800020000000000000008000000000000000000000000000000000000000000000000000400000000000000A935
:2B31E300020000000000000038080000000000000000000000000000000000000000000000000A04000000000008BCAD
:2B320E00040000000000000010000000000000000000000000000000000000000000000000000000000000000008FA7F
:2B32390002000000000000000E020000000000000000000000000000000000000000000000808500000000000008D279
:2B326400020000000000000008000000000000000000000000000000000000000000000000000400000000000088A108
:2B328F00020000000000000074000000000000000000000000000000000000000000000000000704000000000080E52E
:2B32BA00000000000000000008000000000000000000000000000000000000000000000000000004000000000000AF2E
:2B32E500000000000000000030040000000000000000000000000000000000000000000000000A00000000000000F28E
:2B331000000000000000000010000000000000000000000000000000000000000000000000000200000000000080D42C
:2B333B00000000000000000028080000000000000000000000000000000000000000000000008E00000000000080AB7E
:2B336600020000000000000000000000000000000000000000000000000000000000000000000000000000000008ED45
:2B339100020000000000000016020000000000000000000000000000000000000000000000808500000000000088CB9F
:2B33BC00020000000000000010000000000000000000000000000000000000000000000000000400000000000008B810
:2B33E70002000000000000003C100000000000000000000000000000000000000000000000002F00000000000008F343
:2B341200000000000000000000000000000000000000000000000000000000000000000000004000000000000080E3EC
:2B343D00000000000000000008100000000000000000000000000000000000000000000000000200000000000000DD6D
:2B346800000000000000000008000000000000000000000000000000000000000000000000000200000000000000CD62
:2B3493000C0000000000000038020000000000000000000000000000000000000000000000000E04000000000038CFAF
:2B34BE000A0000000000000000000000000000000000000000000000000000000000000000000000000000000018F4CD
:2B34E900000000000000000000000000000000000000000000000000000000000000000000000000000000000080E751
:2B351400800008800008800008800008800008800008000000000020000220000220000220000220000220000280E729
:2B353F00800008800008800008800008800008800008000000000020000220000220000220000220000220000280E7FE
:2B356A00000000000000000020080000000000000000000000000000000000000000000000002002000000000080EF7D
:2B359500000000000000000000000000000000000000000000000000000000000000000000000000000000000080E7A4
:2B35C000000000000002000000000000000000000000000000000000000000000000000000000000000000000080C797
:2B35EB00000802000000000000000000000000000000000000000000000000000000000000000000000000022000C7C2
:2B361600000802000002000020080000000000000000000000000000000000000000000000002202000000022000CD42
:2B364100000000000000000040000000000000000000000000000000000000000000000000000000000000000080A3FB
:2B366C00000000000000000000000000000000000000000000000000000000000000000000000404000000000080E3C8
:2B369700000000000000000000040000000000000000000000000000000000000000000000002000000000000080E183
:2B36C200000000000000000000080000000000000000000000000000000000000000000000000000000000000080EF66
:2B36ED001400000000000000040800000000000000000000000000000000000000000000000000000000000000A09959
:2B371800000000000000000000020000000000000000000000000000000000000000000000000000000000000080E51F
:2B374300000000000000000000000000000000000000000000000000000000000000000000000000000000000080E7F4
:2B376E00000000000000000000000000000000000000000000000000000000000000000000000000000000000080E7C9
:2B379900000000000000000000100000000000000000000000000000000000000000000000000100000000000080E68E
:2B37C400140000000000000000000000000000000000000000000000000000000000000000000000000000000080F353
:2B37EF00000000000000000000000000000000000000000000000000000000000000000000000002000000000080C766
:2B381A000000000000000000000000000000000000000000000000000000000000000000000000020000000000C0833E
:2B3845000000000000000000000000000000000000000000000000000000000000000000000000000000000000A0C5F3
:2B387000000000000000000000000000000000000000000000000000000000000000000000002000000000000080E5A8
:2B389B000000020400000000088008840000000000000000000000000000000000000800000008000000000000008B4D
:2B38C600000008000000000000022000020000000000000000000000000000000000080000008000000000000000ED36
:2B38F100000000000000000000000000000000000000000000000000000000000000000000000000000000000080E745
:2B391C00000000000000000000000000000000000000000000000000000000000000000000000000000000000080E719
:2B394700A0280EA1100AA1108A433884A3100AA110840200000000100441100AA1100EA1100AE12884A2100AA180C380
:2B397200C07597C11DDCC11DDC655886C51DDCC11B06170000000018866118DCC11D96C11DDC617107D71DDCC185CE12
:02399D00FFFF2A
:00000001FF
